:10000000000008308A00D22AFF00030E8312031377
:10001000A1000A08A0008A010408A2007708A30032
:100020007808A4007908A5007A08A6007B08A70034
:10003000831383128B1E1E280B193128220884007B
:100040002308F7002408F8002508F9002608FA001C
:100050002708FB0020088A00210E8300FF0E7F0E78
:1000600009008A110A12132C0A108A100A11820739
:1000700053346D34613472347434203453346834FE
:1000800075347434743465347234203476342034E6
:1000900030342E3434340D340A3400340A108A10CB
:1000A0000A1182076234753469346C347434203434
:1000B0006F346E34203400340A108A100A1182071B
:1000C000313431342D344634653462342D34303497
:1000D000323400340A108A100A1182076134643401
:1000E00063342034763461346C34753465342034B0
:1000F0003D34203425346C3464340D340A340034F7
:100100000A108A100A1182076434693472345F3429
:100110007334743461347434653420343D342034A1
:10012000253464340D340A3400340A108A100A115C
:100130008207703477346D345F34733474346134CF
:100140007434653420343D342034253464340D3423
:100150000A3400340A108A100A1182077234753486
:100160006E345F34733474346134743465342034E1
:100170003D342034253464340D340A3400340A10FC
:100180008A100A1182070D340A345F3465347234E0
:100190007234203473346834753474347434653490
:1001A0007234203463346C346F34733465342034E7
:1001B000743469346D346534643420346F34753488
:1001C00074340D340A3400340A108A100A11EB3EDC
:1001D00003188A0A82000D340A345F34653472349D
:1001E0007234203473346834753474347434653440
:1001F0007234203463346C346F3473346534203497
:10020000633475347234723465346E34743420342B
:1002100074347234693470340D340A3400340A147E
:100220008A100A1182070D340A345F34653472343F
:1002300072342034733468347534743474346534EF
:10024000723420346F34703465346E342034743436
:1002500069346D346534643420346F3475347434E7
:100260000D340A3400340A148A100A1182070D343E
:100270000A345F3465347234723420347334683431
:100280007534743474346534723420346F3470349B
:1002900065346E34203463347534723472346534AA
:1002A0006E347434203474347234693470340D34E0
:1002B0000A3400340A148A100A1182077334743421
:1002C0006F34723469346E3467342034613464348A
:1002D00063342034763461346C34753465342034BE
:1002E0003D34203425346C3464340D340A34003405
:1002F0000A148A100A118207723465346134643436
:100300002034763461346C347534653420343D34B3
:10031000203425346C3464342034663472346F34C1
:100320006D34203465346534703472346F346D3418
:100330000D340A3400340A148A100A1182076D340D
:100340006F3474346F3472345F3470346F34733498
:100350006934743469346F346E3420343D3420345D
:1003600025346C3464340D340A3400340A148A1091
:100370000A11820765346E3463346F346434653433
:100380007234203470346F347334693474346934A3
:100390006F346E3420343D342034253475340D34BC
:1003A0000A3400340A148A100A1182076D346F343B
:1003B00074346F3472345F3470346F34733469342E
:1003C000743469346F346E3420343D342034303426
:1003D000783425344C3478340D3400340A148A10BF
:1003E0000A11F53E03188A0A820065346E346334BC
:1003F0006F3464346534723420346334703473344D
:1004000020343D34203425346C3464340D340A34C3
:1004100000340A108A140A1182076D346F34743460
:100420006F34723420346D346F34763469346E3402
:10043000673420343A34203474347234753465347B
:1004400000340A108A140A1182076D346F34743430
:100450006F34723420346D346F34763469346E34D2
:10046000673420343A342034663461346C34733465
:10047000653400340A108A140A118207313420349A
:100480002D34203467346534743420347434683443
:10049000653420346D346F3474346F3472342034E6
:1004A00070346F3473346934743469346F346E3437
:1004B0000D340A3400340A108A140A1182073234C7
:1004C00020342D34203474346F34673467346C3402
:1004D00065342034703477346D3420342834523409
:1004E0004334323429340D340A3400340A108A1467
:1004F0000A118207333420342D34203474346F349D
:10050000673467346C34653420346434693472344D
:1005100065346334743469346F346E342034283471
:1005200052344234353429340D340A3400340A103C
:100530008A140A118207343420342D342034743460
:100540006F34673467346C346534203472347534F6
:100550006E342F34733465346E3473346534203420
:10056000283452344234343429340D340A340034BB
:100570000A108A140A118207353420342D342034AD
:10058000733468346F347734203449342F344F3423
:100590002034733474346134743465340D340A3463
:1005A00000340A108A140A118207363420342D349C
:1005B00020346F34703465346E34203473346834CE
:1005C000753474347434653472340D340A34003440
:1005D0000A108A140A118207373420342D3420344B
:1005E00063346C346F34733465342034733468345A
:1005F000753474347434653472340D340A34003410
:100600000A148A140A118207383420342D34203415
:10061000733474346F3472346534203470346F340E
:1006200073346934743469346F346E340D340A347D
:1006300000340A148A140A118207393420342D3404
:1006400020347234653461346434203470346F344F
:1006500073346934743469346F346E340D340A344D
:1006600000340A148A140A118207303420342D34DD
:1006700020346D346F3474346F34723420347034F9
:100680006F3473346934743469346F346E340D34B8
:100690000A3400340A148A140A118207613420349F
:1006A0002D34203465346E3463346F3464346534EF
:1006B0007234203470346F34733469347434693470
:1006C0006F346E340D340A3400340A148A140A115B
:1006D0008207623420342D34203463346C34653422
:1006E00061347234203465346E3463346F3464346E
:1006F000653472340D340A3400340A148A140A1131
:100700008207633420342D3420346C346F346F34DA
:10071000703465346E347A3479342034723465340C
:100720006134643420346D346F3474346F34723413
:100730000D340A3400340A148A140A11820764340E
:1007400020342D342034633461346C3463342034E9
:1007500065346E3463346F346434653472342034F9
:100760006334703473340D340A3400340A148A1438
:100770000A118207653420342D34203469347334EF
:1007800020346D346F3474346F34723420346D34EB
:100790006F34763469346E3467340D340A3400347F
:1007A0000A148A140A1182073F3420342D3420346D
:1007B000733468346F347734203474346834693473
:1007C000733420346D3465346E3475340D340A342A
:1007D00000340A148A140A11F03E03188A0A8200AF
:1007E00069346E34763461346C3469346434203462
:1007F000733465346C3465346334743469346F3401
:100800006E340D340A340034091083160910FF3099
:10081000880083120808D500091483160910831272
:100820005508F800003404247808D3002908D200C1
:1008300052085302D4005408003A0319222C013004
:10084000AD00232CAD0154088039003A0319392C2E
:100850005408FF3A013EA9020030031C0130AA02ED
:100860000030031C0130AB020030031C0130AC022D
:10087000472C5408A907003003180130AA0700309C
:1008800003180130AB07003003180130AC07B20B7E
:100890005E2CB30AB10803194F2C0030502C0130E4
:1008A000B100B108031D562C0710572C0714341043
:1008B000340883168700F4308312B2000B118A11BA
:1008C0000A121E28091183160911831209158316AD
:1008D00009118312AC01AB01AA01A9010034B601D0
:1008E00036083420B60A0C1E732C990015303602D7
:1008F000031D702CB60136084E20B60A0C1E7E2C45
:10090000990009303602031D7B2CB60136085C20A5
:10091000B60A0C1E892C990009303602031D862C5C
:100920000D300C1E912C99000A300C1E952C99004C
:100930000A300C1E992C99008A150A12362BB60122
:1009400036083A22B60A0C1EA32C99001C30360237
:10095000031DA02CB60136085B22B60A0C1EAE2C75
:10096000990016303602031DAB2CB60136087622EC
:10097000B60A0C1EB92C99001C303602031DB62C89
:10098000B60136089722B60A0C1EC42C99001C30FA
:100990003602031DC12CB6013608B822B60A0C1E59
:1009A000CF2C990014303602031DCC2CB60136082A
:1009B000D122B60A0C1EDA2C990012303602031D21
:1009C000D72CB6013608E822B60A0C1EE52C990091
:1009D00013303602031DE22CB60136080023B60A96
:1009E0000C1EF02C990014303602031DED2CB601BC
:1009F00036081923B60A0C1EFB2C99001330360258
:100A0000031DF82CB60136083123B60A0C1E062D3C
:100A1000990014303602031D032DB60136084A230F
:100A2000B60A0C1E112D990016303602031D0E2D2C
:100A3000B60136086523B60A0C1E1C2D990013302A
:100A40003602031D192DB60136087D23B60A0C1E89
:100A5000272D990019303602031D242DB6013608C2
:100A60009B23B60A0C1E322D990016303602031D48
:100A70002F2DB6013608B623B60A0C1E3D2D99005F
:100A800015303602031D3A2DB6013608D023B60ABA
:100A90000C1E482D990014303602031D452D0034DC
:100AA0008C1E502D1808A8001A08F800A81C5A2DF2
:100AB0001812181600008A150A123C2B0408C000F0
:100AC000BA1F6C2D2D300C1E632D99008403B909BB
:100AD000BA09B90A0319BA0A3A0EF038BC00BC07C1
:100AE000E23EBD00323EBF003A080F39BD07BD07E8
:100AF000BF07E93EBE00BE07BE07390E0F39BE076D
:100B0000BF07BE0DBF0DBF09BF0D39080F39BF07A5
:100B1000BC0D0730BB000A30BF07BE03031C8C2D81
:100B2000BE07BD03031C902DBD07BC03031C942D01
:100B3000BC07BB03031C982D3B30840007304005E5
:100B400084073F3004020319B92D0008F700031D84
:100B5000AF2D401AB72DC019B12D2030B22D08305D
:100B6000C0003030F70777080C1EB42D9900840AB6
:100B7000A12D0008F7003030F70777080C1EBE2DB6
:100B800099000034B601B7011F151F19C52D831632
:100B90001E088312B6001E08B700B80138086A2084
:100BA000B80A0C1ED12D99000C303802031DCE2D31
:100BB000103084003708BA003608B9005E250D30C1
:100BC0000C1EE02D99000A300C1EE42D99008A15A8
:100BD0000A12842BAF080319EF2D0030F02D0130DD
:100BE000AF00AF08031DF62D0711F72D07153411BF
:100BF00034088316870083128A150A12882BAE08E0
:100C00000319042E0030052E0130AE00AE08031D7E
:100C10000B2E86120C2E86168316861283128A15C8
:100C20000A128C2BB0080319172E0030182E013031
:100C3000B000B008031D1E2E06121F2E06168316C6
:100C4000061283128A150A12902B3B08F8013A0209
:100C500003182D2E3A08F700392EF7010830BC0092
:100C6000BA0DF70D3B0877020318F700F80DBC0B1F
:100C7000302E00342030F8003708F700B71F462E1A
:100C8000F709F70A7708B7002D30F80078080C1E2E
:100C9000472E99003818652EB818792E3708BA00F3
:100CA0006430BB0025267708B70078083030031D74
:100CB0005E2E3819652EB8192030602E3811B81103
:100CC000F80778080C1E622E99003708BA000A301F
:100CD000BB0025267708B70078083030031D742E36
:100CE0003819792EB8192030F80778080C1E762E9E
:100CF00099003030B70737080C1E7C2E990000345D
:100D00000E30B6002D300C1E832E9900B60B822EAD
:100D10000D300C1E892E99000A300C1E8D2E990064
:100D2000B60136088020B60A0C1E942E99000C30AD
:100D30003602031D912E2E08B7000C30B8003A265B
:100D40000D300C1EA12E99000A300C1EA52E990004
:100D5000B60136089520B60A0C1EAC2E99000C3050
:100D60003602031DA92E2F08B7000C30B8003A2612
:100D70000D300C1EB92E99000A300C1EBD2E9900A4
:100D8000B6013608AA20B60A0C1EC42E99000C30F3
:100D90003602031DC12E3008B7000C30B8003A26C9
:100DA0000D300C1ED12E99000A300C1ED52E990044
:100DB0000E30B6002D300C1EDB2E9900B60BDA2E4D
:100DC0000D300C1EE12E99000A300C1EE52E990004
:100DD0008A150A12942B3B30840000080319FF2E59
:100DE0000130F800F701F70BF32EF80BF22E4A3022
:100DF000F700F70BF92E00000000800BF02E0034F6
:100E00008101F430B200B3010034B608031D702F25
:100E10001F151F19092F1E08FA0083161E088312BA
:100E2000B7001E08B800B808031D1A2F3708C73CC2
:100E30000318DD2FAE01AE08031D202F8612212FCF
:100E4000861683168612831206168316061214302F
:100E50008312BB00EB2683160616831200271F158C
:100E60001F19302F1E08FA0083161E088312B700C0
:100E70001E08B800B808031D412F3708C83C0318E6
:100E80006B2F3308033C0318552FB7013708BF20D9
:100E9000B70A0C1E492F990020303702031D462F38
:100EA00006128316061283126B2F83160616831200
:100EB000061A6A2F0612831606128312B701370824
:100EC000E420B70A0C1E622F990023303702031D5D
:100ED0005F2F6B2F2F2F0612831606128312DD2F22
:100EE0001F151F19712F1E08FA0083161E08831282
:100EF000B7001E08B800023C0318852FFF3A031DF7
:100F0000842F3708203C031CDD2F0130AE00AE08D3
:100F1000031D8C2F86128D2F861683168612831240
:100F200006168316061214308312BB00EB268316B6
:100F30000616831200271F151F199C2F1E08FA0082
:100F400083161E088312B7001E08B800033C031C5A
:100F5000D92F031DAF2F37081F3C031CD92F33088F
:100F6000033C0318C32FB70137080F21B70A0C1E23
:100F7000B72F99001F303702031DB42F06128316B6
:100F800006128312D92F831606168312061AD82F3B
:100F90000612831606128312B70137083321B70AE7
:100FA0000C1ED02F990022303702031DCD2FD92FD0
:0C0FB0009B2F06128316061283120034D9
:101000001F151F19012883161E088312B6001E081B
:10101000B700B80138088A115A218A15B80A0C1E7F
:101020000F28990014303802031D0A28103084005C
:101030003708BA003608B9008A115E258A150D30C6
:101040000C1E202899000A300C1E2428990037080D
:10105000B80003178D018F010313380803178C00A4
:1010600083168C130C15831203130B08F7008B13D4
:101070005530831603178D00AA308D008C1483120F
:101080000313831603178C1C48288312031341286B
:101090000C117708831203138B043608B800013053
:1010A00003178D008F010313380803178C00831674
:1010B0008C130C15831203130B08F7008B13553098
:1010C000831603178D00AA308D008C14831203132E
:1010D000831603178C1C6F288312031368280C11C6
:1010E0007708831203138B048A150A12A22B0317A5
:1010F0008D018F0183168C130C1483120C080313BB
:10110000B800013003178D008F0183168C130C1467
:1011100083120C080313B9003808B7003908B60069
:10112000B80138088A1178218A15B80A0C1E962849
:1011300099000D303802031D9128103084003708C3
:10114000BA003608B9008A115E258A151030B90038
:1011500039088A1178218A15B90A0C1EAD28990020
:101160001E303902031DA8288A150A12A42BF70184
:10117000F801F901FA01CD01CE01CF01D0014C08EF
:101180004B044A0449040319F5282030D100031008
:10119000C50DC60DC70DC80DCD0DCE0DCF0DD00D93
:1011A0004C085002031DDE284B084F02031DDE28A9
:1011B0004A084E02031DDE2849084D02031CEF2891
:1011C0004908CD024A08031C4A0FCE024B08031CF3
:1011D0004B0FCF024C08031C4C0FD0020314F70D29
:1011E000F80DF90DFA0DD10BC72800004D30840021
:1011F00000340408BF00BE1F0C292D300C1EFE2831
:101200009900BB09BC09BD09BE09BB0A0319BC0A88
:101210000319BD0A0319BE0A3B30C4009A30C3004B
:10122000CA30C200C1010A30C0003E08C8003D08F3
:10123000C7003C08C6003B08C5004408CC00430872
:10124000CB004208CA004108C900B7200008BB0013
:10125000840A0008BC00840A0008BD00840A000853
:10126000BE00FD308407F708031D48294008013AF5
:10127000031948293F08031949290F394002031966
:10128000432903184F29F0303F1B0030F70049294C
:10129000BF013030F70777080C1E4C29990044082D
:1012A000C8004308C7004208C6004108C500CC0179
:1012B000CB01CA010A30C900B7207A08C4007908F6
:1012C000C3007808C2007708C100C00B152900349C
:1012D000B60136088A119B218A15B60A0C1E6E29A2
:1012E000990011303602031D6929413084002C0811
:1012F000BE002B08BD002A08BC002908BB00F9204D
:101300000D300C1E812999000A300C1E8529990088
:101310008A150A12A62B3918A829B918BE29380827
:10132000BA006430BB008A1125268A157708B800F8
:1013300078083030031DA1293919A829B91920309E
:10134000A3293911B911F80778080C1EA5299900AD
:101350003808BA000A30BB008A1125268A1577089A
:10136000B80078083030031DB9293919BE29B919D8
:101370002030F80778080C1EBB2999003030B807D8
:1013800038080C1EC12999008A150A12E4290B0895
:101390000B058B13A0008A1104248A1520088B04E6
:1013A0007808B600B70137088A11B6218A15B70A3E
:1013B0000C1ED829990013303702031DD329360893
:1013C000B8000C30B9008B290D300C1EE5299900AE
:1013D0000A300C1EE92999008A150A12A82BB81B9D
:1013E000022A0F30F700370EF7050A30770203188C
:1013F000FC293030F707FE293808F70777080C1E5C
:10140000FF2999000F30B7050A30370203180A2A5E
:1014100030300C2AB8133808B70737080C1E0E2ACC
:10142000990000348C1A3F2AB60136088A11D2215D
:101430008A15B60A0C1E1A2A990013303602031DAB
:10144000152A2C08B7005730B800EF212B08B70039
:101450005730B800EF212A08B7005730B800EF2105
:101460002908B7005730B800EF210D300C1E362A7E
:101470009900C830BB008A11EB268A15122A8A15FA
:101480000A12AE2BAE010130B000AE08031D4A2A8D
:1014900086124B2A8616831686128312B008031D05
:1014A000532A0612542A0616831606120230831295
:1014B000BA00FA30BB008A11EB268A15BA0B592AFA
:1014C0008A1162248A150430BA00FA30BB008A11EE
:1014D000EB268A15BA0B652A2C08B9002B08B80030
:1014E0002A08B7002908B600B001B008031D7A2AFF
:1014F00006127B2A0616831606128312BA013A08D0
:101500008A11EE218A15BA0A0C1E842A99000E301F
:101510003A02031D7F2A413084003908BE00380892
:10152000BD003708BC003608BB00F9200D300C1E8A
:10153000972A99000A300C1E9B2A99008A150A12D4
:10154000B02BAD080319BA2AB60136088A11092250
:101550008A1500380319B12AB60A0C1EAD2A990063
:10156000A52A0D300C1EB22A99000A300C1EB62A8C
:101570009900CF2AB60136088A1121228A1500382F
:101580000319C72AB60A0C1EC32A9900BB2A0D30BC
:101590000C1EC82A99000A300C1ECC2A99008A1504
:1015A0000A12B22B84011F3083059F30840007305C
:1015B0008000A801193083169900263098009030D9
:1015C00083129800AE01AF01B001B101B201B301C5
:1015D000FF30B400AE01AF01B0018A1162248A1558
:1015E000AE08031DF52A8612F62A86168316861281
:1015F0008312AF08031DFE2A0711FF2A07153411B5
:101600003408831687008312B008031D092B0612C5
:101610000A2B061683160612F4308312B2008101DB
:101620000330F700F71D1C2B073081018130840047
:101630000008C0390F388000640081308400000841
:10164000C039770480008B16C0308B048430831639
:101650009F0083121F083839C1389F000030F800FE
:101660001F08C73978049F008A116F2C8A158A11C8
:101670009F248A158A11502D8A157808B5003508DF
:10168000F700313035020319822B3230770203190B
:10169000862B3330770203198A2B343077020319F3
:1016A0008E2B353077020319922B363077020319CF
:1016B000962B3730770203199C2B383077020319A9
:1016C000A12B393077020319A32B3030770203198D
:1016D000A52B613077020319A72B6230770203191B
:1016E000A92B633077020319AD2B643077020319FD
:1016F000AF2B653077020319B12B3F307702031906
:10170000B32BB72B8A11C22D8A15C42B8A11EA2D4F
:101710008A15C42B8A11FF2D8A15C42B8A11122E0B
:101720008A15C42B8A11802E8A15C42B0130B6006D
:101730008A1105278A15C42BB6018A1105278A1537
:10174000C42B0028C42B7728C42B6829C42BC72995
:10175000C42B8A1162248A15C42B122AC42B422A54
:10176000C42BA12AC42B8A119F248A15C42BB6012D
:1017700036088A11E9238A15B60A0C1EBD2B99007A
:0C17800013303602031DB82B3A2B630017
:02400E00F13788
:00000001FF
